:020000040800F2
:10500000201A0020D5500008ED820008157B00080A
:105010000000000000000000000000000000000090
:105020000000000000000000000000008D8F00085C
:10503000000000000000000045880008B99000084A
:10504000E7500008E7500008E7500008E750000864
:10505000E7500008295B0008E7500008E750000807
:1050600000000000E7500008515A0008E75000080F
:10507000E7500008697F000800000000E7500008C2
:1050800000000000E75000080000000000000000E1
:10509000E750000800000000E7500008E750000853
:1050A000E7500008E7500008E7500008459800085E
:1050B000E7500008E7500008000000000000000072
:1050C0000348854600F060FC0048004771A60008D0
:1050D000201A00200448804704480047FEE7FEE706
:1050E000FEE7FEE7FEE7FEE755910008C150000825
:1050F00030B50B46014600202022012409E00D4670
:10510000D5409D4205D31D469540491B25469540F7
:1051100040191546521E002DF1DC30BDF0B51FB40C
:105120000646002082B005464024019100901BE015
:10513000019922460F46304600F04EFB049A059B2B
:10514000801A994110D310461946224600F034FBCC
:10515000361A8F410197224601200021009F00F05E
:105160002BFB38184D4100902046641E0028DFDCE0
:10517000019B00982946324607B0F0BD03460B4319
:105180009B0703D009E008C9121F08C0042AFAD2FD
:1051900003E00B780370401C491C521EF9D2704783
:1051A000D2B201E00270401C491EFBD270470022BF
:1051B000F6E710B513460A4604461946FFF7F0FF16
:1051C000204610BD30B504460020034600E05B1CBD
:1051D000934203D2E05CCD5C401BF8D030BDF8B503
:1051E00002464A40D40F42004B0052085B089A42E4
:1051F00002D20246084611464A0023D0C30D4A0097
:10520000DDB2120EAD1A202D35DA49020126490A07
:10521000F6058A19002C00D0524220214F1B11465E
:10522000B9402A411018C20D9A4221D0002C17D043
:10523000012D08DCDA05801AD20F8019D207DBB203
:1052400000F0F6FAF8BDDA05801A012340001B06CB
:10525000C01880185A428018CA0F1043490007E04E
:105260004908C2071143DA05801A801940088018DE
:1052700000F0D6FAF8BD61000122511A001BF7E7D1
:105280000122D2075140AAE70122D2075040A6E7E7
:1052900070B502464A40D50F40004A00ED0740086D
:1052A0005208002814D0002A12D0C40DD30D410298
:1052B0000120C0055202490A520AE41A09181218BC
:1052C0007D34914201D3641C00E04900002C01DAD6
:1052D000002070BD0023914201D3891A0343400886
:1052E00049000028F7D100290AD0914202D10121BA
:1052F000C90705E0914201D2012101E00121C94322
:10530000E005C018401900F08BFA70BDF0B50746F3
:105310000846584087B0C00F049048000E46590018
:1053200040084908BC1A884105D2384631461E4615
:1053300017460B4602465800400810434CD0300D2B
:10534000039040055900400D490D0590401A029008
:10535000402872DA18030121000B09050843019067
:1053600004980092002805D00199524200208841FB
:1053700000920190029840210A1A0199009800F0C9
:105380001BFA05460C466B4607CB00F036FAC019EF
:105390007141039A0E0D0023D71756401A467A40E2
:1053A000164344D0049A002A2DD0029A012A039A67
:1053B00015DC1205C01A914101263605001C714109
:1053C000D20F059ED2070093019202962A462346E9
:1053D00000F074FA07B0F0BD38463146FAE716051A
:1053E000224A0F46B218C01AB74101210905001C14
:1053F0004F4100187F41114618187941E20F1043C0
:105400006D19644113E0E2076D0815436408C20793
:105410001443039A01261205C01A91413605001C57
:105420007141CE07400830434908C01851412A460F
:10543000234600F036FACDE7FFE70498012240004A
:10544000C117121A00238B4104983146C417381A29
:10545000A141EEE730B40124E407634030BC55E7D6
:1054600030B40124E407614030BC4FE70000E0FFA6
:10547000F0B51FB488B00B990998002448400999E9
:10548000C00F490049080991C0070B9900904900D5
:1054900049080B9109990898A64608431CD00B9916
:1054A0000A98084318D0099801244000420D48008A
:1054B000410D099824050003000B204309900B9827
:1054C0000003000B20430B9050181C494018002289
:1054D00001901446104605E0002001460DB0F0BDD5
:1054E000032801DA034600E003239C46C11A0AAEF2
:1054F0000AE05F0008ADED5B4F00F75B7D430027DE
:10550000AA187C41491C5B1E6145F2DD410004ABD9
:105510005A522104120C0A43240C401C0828DFDBD9
:10552000019802900099704601910090059B049AA1
:105530000799069800F0C2F9D0E700000DFCFFFFC4
:10554000F0B50C465C4085B0E40FE40703944C00D2
:1055500000266408590094464908024602962243F0
:1055600021D062460A431ED06200570D4A000E0346
:105570002303550D012402462C492405781B1B0BDF
:10558000360B401823432643614600901C46501AB0
:10559000B44103D30098401C009002E09218009898
:1055A0005B41002803DA0020014605B0F0BD002071
:1055B000012109050746864611E064461D46141B75
:1055C000B54106D36546521BB341744607430C43AD
:1055D000A646CD0740084908284392185B41054676
:1055E0000D43EAD11046184313D060461946504087
:1055F0007140084306D06046101AB34106D201221A
:10560000002306E000220123DB0702E00122D2434F
:105610005310009874460105381C6141029C039D9B
:105620000019694100F03DF9BFE70000FD030000EB
:10563000C217C10F504010B54018CA079623002169
:1056400000F0F6F810BD10B500229623114600F0C8
:10565000EFF810BD0EB5C217C10F5040CA07401871
:105660000021054B0293019200910A460B4600F07F
:1056700025F903B000BD0000330400000EB5054954
:105680000291002100910A460B46019100F016F9A3
:1056900003B000BD33040000410040020122400A73
:1056A000D205090E80187F2901DA0020704796295B
:1056B00003DC9622511AC8407047963988407047DB
:1056C00070B5CD0F4A0009030123090B1B051943CF
:1056D0000B4BED070024520D9A4201DA002070BDF9
:1056E000074B34339A4203DC9A1A00F075F802E053
:1056F0000449511888402C43F1D0404270BD00004D
:10570000FF030000CDFBFFFF4A0009030123090B43
:105710001B051943094B10B5520D9A4201DA0020BE
:1057200010BD064B34339A4203DC9A1A00F054F849
:1057300010BD03495118884010BD0000FF03000050
:10574000CDFBFFFFC20FD207400040080BD0C10DB8
:105750000723DB01C91840020905400A1143C208AA
:10576000400711437047002001467047CB0FDB070D
:10577000490010B5490802460A4307D00A0D07241C
:105780000903E401090B121B002A01DC002010BDF3
:10579000C900440F0C43C100E018D205801800F086
:1057A0003FF810BD0122D207002800DB101A0029A3
:1057B00000DB511A8142704710B5202A04DB0146F4
:1057C000203A9140002010BD914020239C1A0346AE
:1057D000E3401943904010BD10B5202A04DB084671
:1057E000203AD040002110BD0B46D340D0402024A9
:1057F000A21A91400843194610BD10B5202A06DBB5
:10580000CB170846203A1041C1170B4306E00B4660
:105810001341D0402024A21A91400843194610BDDC
:10582000002904DA401C490001D1400840007047BB
:1058300070B40024050C05D11024000402D1002905
:1058400021D01124050E01D100020834050F01D129
:105850000001241D850F01D18000A41C002801DB5C
:105860004000641C002908D020252E1B0D46F54061
:10587000A14000D001212943084301061B1B000A57
:10588000DB1D02D5002070BC7047DB05181880189E
:105890000029F8DA401C4900F5D170BC40084000EE
:1058A000704710B5002B08DA0024401C61419218A3
:1058B0005B411A4301D14008400010BDF0B51FB450
:1058C00082B005460C0003D0084604F07BF802E0E5
:1058D00004F078F820300246009021462846FFF771
:1058E0006BFF049B059A04460F4618431143084377
:1058F00014D0184610431BD0009840210A1A1846AD
:105900000599FFF769FF05460E46009A0599049828
:10591000FFF752FF084305D0012004E02046394636
:1059200007B0F0BD0020C11705430E432C43374399
:1059300000990E986305401A7905E40A00220C4389
:10594000FD0A0A3002D500200146E9E701051019D9
:1059500069410C9C0D9D00196941FFF7A2FFDFE72B
:1059600010B5002904DB0124E40740428C412146A4
:10597000002B04DB1C460123DB075242A341994262
:1059800000D1904210BD0000064C0125064E05E0F6
:10599000E36807CC2B430C3C98471034B442F7D350
:1059A000FFF792FBE4A9000804AA000838B50446F2
:1059B000064805490068FFF79BFB604300E0401E76
:1059C00000900028FBD138BD40420F001C01002090
:1059D000F8B50446006881688907890F012902D15A
:1059E0000168C90722D18168114A1026114001259A
:1059F00000290ED18168294381600120FFF7D6FF7D
:105A000000F078FF07460CE000F074FFC01B0A2886
:105A100007D9606D30436065A06D2843A065012003
:105A2000F8BD20680068C043C007EDD10020F8BD74
:105A30001700008010B500231A4603E0845CE318C9
:105A40009BB2521C8A42F9D3D84380B210BD0000E9
:105A500010B5034800F00EFD024800F00BFD10BD2C
:105A6000C01500207815002030B5446C1C252C4052
:105A70000125A540046C6560046863608368102B91
:105A8000036803D099600068C26030BD9A60006806
:105A9000C16030BD1449012048720A4602205E32BE
:105AA000507203203C3A507204200E3A50720F4854
:105AB0000D4B0078087022310870203108770C49AE
:105AC0005A1C0878587149789971233318715971A3
:105AD000203318775977107551751A461E32107594
:105AE000517510765176704750110020D800002073
:105AF000F400002010B503F021FA202003F0D2FAC0
:105B0000012004F00FFB002003F0CCFA044804F05D
:105B1000ADF9044804F05CFC002004F091FC10BDD9
:105B2000C000002083800000F8B505200121000797
:105B300000F0D0FE0025184C002800D06560174EFC
:105B40000221304600F0C6FE00281DD10120207041
:105B50001348808F00280ED00127BF02002239464B
:105B6000304600F0C0FE0A2004F032F90122394626
:105B7000304600F0B8FE0B48656000880A214843B3
:105B80000949088003F070FE012000F0DBFD0220CF
:105B900000F0D8FDF8BD00000C010020000400500A
:105BA000500D0020E6000020F200002070470000A9
:105BB00010B5084900224A6107494B684C15234338
:105BC0004B604B68082423434B60C009C00102604E
:105BD00010BD000008160020002002407FB50025FF
:105BE0000C460646039500F07DFDE009029003A9EE
:105BF00001960095684600F00DFD002804D000F0E5
:105C000045FD002004B070BD00F040FD0120F9E723
:105C100010B5002302E0C45CCC545B1C9342FAD361
:105C200010BD000010B5214A00219069C30520482D
:105C300004D54169022319434161911593699B057C
:105C400005D54369012423434361630219439369E2
:105C50005B0505D54369082423434361E3011943E8
:105C600093691B0505D543690424234343616302FB
:105C7000194393699B0405D5436910242343436169
:105C80006302194393699B0304D5446920231C4391
:105C9000446119439369DB0305D5436940242343D9
:105CA0004361A0020143916110BD00000020024049
:105CB0000816002070B5054600F01CFE0646184C7C
:105CC0000AE0681C08D0002D04D000F013FE801BF1
:105CD000A84201D9032070BDA069C007F1D1A06915
:105CE000800701D50220A061A069C00511D4A06978
:105CF00080050ED4A06940050BD4A069000508D426
:105D0000A069800405D4A069800302D4A069C003FF
:105D100003D5FFF787FF012070BD002070BD000094
:105D200000200240F8B51746002605460C4600F054
:105D3000D9FC09E029460220226800F0B5FC0028C1
:105D400004D1241D2D1D361DBE42F3D300F09EFC50
:105D5000BE4201D20020F8BD0120F8BD10B50849AF
:105D600002460020054B497905E044001C5B944243
:105D700003D0401CC0B28842F7D310BD7812002077
:105D80005800002010B500F0AAFD10BD10B509485C
:105D900000F0D2FF80B2FFF771FC074A074BFFF714
:105DA00067FB0022064BFFF7CBFBFFF7ADFC80B291
:105DB00010BD000070140020F853E3A59B843E4002
:105DC00000408F4070B5314D2F48297F0175697FA4
:105DD00041752F490A780276497841762A4905208B
:105DE000133148720A2004F0E3FA7D20C00004F069
:105DF000F9FA2549002213310C2004F0C3FB0021DD
:105E00000C2004F0D1FB022004F022FB214C0021E5
:105E10000F2004F04DFA2042E862F8D0E86A411CF5
:105E200030D040042DD58122D20100210F2004F072
:105E30007EFB0021102004F03BFA41061248490E77
:105E40000022633004F06AFA0F4C6334607A05284C
:105E500017D102220E49601DFFF7B4F9002810D1B6
:105E60000A48A67C6E710422611C4030FFF786F957
:105E700021461331084672005130FFF77FF90320A5
:105E8000287070BD02F056FAB111002058000020B1
:105E9000F400002000D0272410B5084800F096FA3E
:105EA0000A21064800F032FA044800F01DF9800586
:105EB00003D5024800F01AF980B210BD1414002076
:105EC000F8B52F4D00220121284600F00CFDFFF708
:105ED000E3FFFFF7B8FB2B4E3146FFF7D9F92A4C09
:105EE0000122A0601146284600F0FDFC2749A06869
:105EF000002588423EDB2078254F002815D02570EC
:105F0000FFF7CAFFFFF79FFB3146FFF7C1F9A0601B
:105F1000FFF718FC00223B46FFF79CFA00221D4BBE
:105F2000FFF7A6FAFFF722FC6060A068FFF70AFC03
:105F300000223B46FFF78EFA174A184BFFF798FAF4
:105F400006460F466068FFF7FDFB134A144B5242AA
:105F5000FFF78EFA32463B46FFF7D8F9FFF706FC0B
:105F600010496060884201DD616004E0FF21C905DD
:105F7000C84200D365606068FFF78EFBC0B2F8BD11
:105F80000004005000401B4430000020000060402E
:105F900000000C4000E064403333333333B330400F
:105FA000CCCCEC3F0000C842F8B50546044640356D
:105FB000287C0026012808D00120287420688168E8
:105FC0008907890F01290ED101E00220F8BD01687F
:105FD000C90708D0606D20210843606501260020B4
:105FE00028743046F8BD616DFF22013291430222D0
:105FF00011436165C1688907890F0091C1688908EB
:106000008900C1602068816892071143816000F0B7
:1060100071FC07460EE000F06DFCC01B0A2809D990
:10602000606D0221884310210843606500202874B8
:106030000120F8BD206880680028ECDB2068C1687A
:10604000009A1143C160606D80088000401C60654B
:10605000C5E70000F8B506460D464036317C0129FB
:106060000DD00121317401688A68520709D5416D4C
:10607000202211434165002030740120F8BD022028
:10608000F8BD174B6A68D80547109A42154C8A6AC2
:106090002B6812D05B035B0B1A438A6229684903A1
:1060A00005D5A1680143A1600A20FFF77FFC28689D
:1060B000800312D5A06838430EE05B035B0B9A4364
:1060C0008A622968490302D5A1688143A1602868D2
:1060D000800302D5A068B843A06000203074F8BDEA
:1060E0000110000000270140406D70470068006CFF
:1060F0007047000070B5040006D0606D264600258C
:106100004036002802D006E0012070BDA565357438
:10611000204600F0D3F8606DC00603D4216888687B
:10612000400705D5606D1021084360653574EBE7C5
:10613000606DFF220132904302221043606588683F
:106140008207920F5B48012A02D10A68D2072BD13D
:10615000032362689B079A4205D05B429A4202D0B1
:106160005B009A4209D10A69920092080A6121688B
:106170000A6963681A430A610CE00A69920092088E
:106180000A6181680F22920491438160816862688C
:10619000114381602168CA6818239A43CA60216844
:1061A000CA68A3681A43CA608168012252069143F3
:1061B00081608168A28E52061143816020688168E7
:1061C000C90004D48168012212071143816020684C
:1061D000C168394A1140C1602069E168022825D0B0
:1061E00000200143204620300278037B52035B00ED
:1061F0001A431143226B1143A26992031143E269CE
:10620000D20311432268D3681943D160616A0A46F8
:10621000FF3AC23A05D0A26A11432268D3681943F3
:10622000D16042780121012A02D00BE00420D8E796
:106230000078002823D0606D202210436065A06D97
:106240000843A065E06B012820681FD00169C907D9
:1062500003D0016949084900016120684169C90802
:10626000C900416120684169A26B11434161A56584
:10627000606D80088000401C6065002070BD206853
:10628000C26801231B041A43C260DBE70269FF23D3
:106290009B009A43026120680269236CA66C1A4332
:1062A000636C33431A430261206802690A43026146
:1062B000D3E70000002701401902FEFF10B586B0A9
:1062C000044614216846FEF772FF0E492068884292
:1062D00016D10D48416B421511434163C16A012239
:1062E0001143C162C06A69461040059002200090C7
:1062F00003200190002002900520000700F02EFAF4
:1063000006B010BD0024014000100240F8B504465C
:106310004069254640350E4608280BD02068C068E5
:10632000C00709D0606D20210843606500202874F3
:106330000120F8BD082700E00C2700F0DBFA0090F0
:1063400011E0701C0FD0002E05D000F0D3FA009998
:10635000401AB04207D9606D0421084360650020EF
:1063600028740320F8BD206800683842E9D0606DC9
:1063700001214902084360652068C16809058A0F48
:106380000C21002A1BD12022125D002A17D102689D
:10639000120714D5826853070122002B08DB4368DB
:1063A0008B434360606D130298431043606506E0C1
:1063B000606D202318436065A06D1043A065A0693F
:1063C000002801D1206801600020F8BD70B50446A6
:1063D000216800208968490721D425464035297C59
:1063E00001291CD001212974E169012904D020462A
:1063F000FFF7EEFA002811D1616D0A4A1140FF2221
:106400000132114361650021A165297422681C21B4
:10641000116021688A6804231A438A6070BD0220D3
:1064200070BD0000FEF1FFFF70B500240146203171
:106430004A79022A03D00421C163012418E00268CA
:1064400013680E25AB431360026813685B085B009A
:106450001360436C1C221340012215469D40036CBF
:106460005D604A7100220A71816B002900D0884763
:10647000204670BDF0B4016C0D6801680C68466C74
:106480001C2304221E401746B7402F420ED0670738
:106490000CD50C68A40602D40C6894430C60416CC3
:1064A00019408A40016C4A60016B1AE00227B7402C
:1064B00002462F402032002F17D0A70715D50C68B1
:1064C000A40605D40C680A25AC430C600121517167
:1064D000446C02211C40036CA140596000211171E1
:1064E000C16A002918D0F0BC08470827B7402F42DE
:1064F00012D0240710D50C680E25AC430C60446CF8
:1065000001211C400B46A340046C6360C1635171C0
:1065100000211171416BE4E7F0BC704770B50400D5
:106520003CD01F48256814212818FEF7E1FD8000A3
:1065300060641C48206402212046203002464171DC
:1065400029681948E3680140A0686669184323690F
:1065500033431843A3691843E3691843236A184374
:10656000084328600121A0688903884210D00D48A3
:106570008030836A656C1C210D400F26AE40B3430A
:106580008362656C63680D40816AAB400B43836234
:106590000020E06301215171107170BD012070BDB8
:1065A000F8FFFDBF000002400F80FFFFF8B5044672
:1065B0008C46203001790025012909D00126067179
:1065C00041790027012905D0077102252846F8BD29
:1065D0000220F8BD02214171E76320680168490883
:1065E0004900016061462046FFF73EFA206B002813
:1065F0002068016801D00E2205E004229143016069
:10660000206801680A221143016020680168314353
:106610000160DBE7F8B51A4E0546307C0F460128CD
:1066200007D0012030741748FFF744FB010002D067
:1066300021E00220F8BD0020C04338606C6814E0FF
:106640002046FFF7B5FA0F48FFF734FB01460E4826
:10665000426808239A434260426843159A43426065
:10666000002901D03C6006E08034A8686A68C00157
:106670008018A042E4D8002030740846F8BD00001D
:106680000816002050C30000002002400548416861
:106690000222114341604168012211434160002000
:1066A0007047000000200240F8B50C4C1646207CD4
:1066B0000F46012808D0012020740948FFF7FAFA94
:1066C0000025002802D006E00220F8BD65613E608A
:1066D0000348FFF7EFFA2574F8BD00000816002004
:1066E00050C3000011484168C9070BD0EFF3108177
:1066F00072B60F4AC2600F4AC26081F310884168C7
:10670000C9070ED1416889070DD5EFF3108172B624
:10671000094A0261094A026181F3108840688007D2
:1067200001D5012070470020704700000020024082
:10673000EFCDAB8905040302BFAE9D8C1615141373
:106740007047000010B504494A69024202D048610E
:10675000FFF7F6FF10BD000000040140F8B500236C
:106760000124A2E027469F403A4070D04D68022D98
:1067700001D0122D14D1DD08AD002D1800952D6A21
:106780005E07AC46F50E0F26AE46AE406546B543F5
:10679000AC460E697546AE4065462E43009D2E629E
:1067A0004D68012D05D0022D03D0112D01D0122DE1
:1067B00016D185680326AC465D00AE46AE40654600
:1067C000B543AC46CE687546AE4065462E438660FE
:1067D00046680D79BE43ED06ED0F9D40354345609B
:1067E00006685F000325BD40AE46AE430D79B44652
:1067F000AE07B60FBE4065462E430660C6687546B6
:10680000AE438D68BD403543C5604D68ED004BD546
:10681000294D6E6B26436E639E08284DB600751990
:10682000AC46AD689E07360F0F27B740BD4305271E
:106830003F07B84201D1002715E0214FB84201D1EE
:10684000012710E01F4FB84202D102270BE02BE0D6
:106850001D4FB84201D1032705E01C4FB84201D1BA
:10686000052700E00627B7402F436546AF60184D67
:106870002E684F689643FF0300D516432E606E685E
:106880004F689643BF0300D516436E60AE684F68ED
:106890009643FF0200D51643AE60EE684F689643FC
:1068A000BF0200D51643EE605B1C0A681546DD404A
:1068B00000D057E7F8BD0000001002400000014082
:1068C0000004005000080050000C0050001C005054
:1068D000000401400069084000D00120704742696F
:1068E0004A4042617047002A01D08161704781624D
:1068F0007047000001480068704700001801002040
:1069000002480168491C016070470000180100201E
:1069100010B5084800240168402211430160204658
:1069200000F00AF8002801D0012401E000F030FA5C
:10693000204610BD0020024070B5054609487D2163
:106940000024C9000068FEF7D3FB00F0C5FE002854
:1069500001D0012404E000222946501E00F038FA3C
:10696000204670BD1C01002070477047F8B5664C8A
:10697000E078401CE07001206071208B401C208377
:106980006248008802F040FB6148C088FEF75BFE69
:106990006049FEF77DFC604D2968FEF720FC286009
:1069A000A078002500280BD102215C48FFF792FF58
:1069B00002005B495B4819D00022FFF794FF256372
:1069C000594E01203768C005874257DB608AFEF7C1
:1069D0003AFE01467F20C005FEF75AFC3946FEF715
:1069E00053FC306051480221017049E00122D1037B
:1069F0004C48FFF778FF4648C088FEF724FE45491B
:106A0000FEF746FC216BFEF7EAFB4949206388420A
:106A1000D6DD3F480127F926403000900A21304654
:106A2000FEF766FB002903D13D493E48FFF7AAF96E
:106A300002213A48FFF74EFF002801D0002701E06D
:106A4000002F12D102213548FFF744FF00280CD156
:106A500003F0D8FE00990120888003F033FF642002
:106A600003F0B6F934493348C8600A2003F0B0F99E
:106A70003046761EF6B20028D0D1A1E72B4805702B
:106A800002212648FFF726FF002809D02563224E61
:106A90002A4937682A488F4214DD0121017012E02B
:106AA0001B48C088FEF7CFFD1A49FEF7F1FB216BAA
:106AB000FEF795FB234920638842E8DB1E491D4809
:106AC000C860E4E705701248408F401EFEF7B0FD35
:106AD0003946FEF767FE06D8A079002803D01A4988
:106AE0000120087001E0184805700948408FFEF742
:106AF000AAFD3168FEF756FE04D2A079002801D025
:106B000003F044FEF8BD0000D40000207200002015
:106B1000500D002000007A441001002000040050B5
:106B200000800000000000501401002069000020D7
:106B3000000040400400FA0500ED00E00000F042D3
:106B40005E0000200000A0406B000020704770B580
:106B500005000DD002202C462034A073284601F0F9
:106B60000BFA284600F0BEF80020A073607370BDD9
:106B7000012070BD7047704710B504460068016879
:106B8000C943C90708D18168C943C90704D1012194
:106B900041602046FFF7EAFE20680168C943890783
:106BA00008D48168C943890704D402214160204682
:106BB000FFF7DAFE20680168C943490708D48168F5
:106BC000C943490704D404214160204600F0DEF89F
:106BD00020680168C943090708D48168C9430907C7
:106BE00004D4082141602046FFF7B0FF2068016807
:106BF000C943C90608D48168C943C90604D4102111
:106C000041602046FFF7B1FE20680168C94389064C
:106C100008D48168C943890604D4202141602046F4
:106C2000FFF7A9FF20680168C943490608D48168B5
:106C3000C943490604D4402141602046FFF79AFF2A
:106C400010BD0000F8B5040005D025462035A87B0E
:106C5000002802D006E00120F8BD0020687320461D
:106C600000F052F80220A8732068C2688446636866
:106C7000012B04D00120A16AC005814201D11E2050
:106C8000824315486169814201D01448024014488A
:106C9000A668024018463043676A266A3E4330437E
:106CA000A66A30431043012B03D00122D20596423D
:106CB00003D12369E2681A431043074A914205D081
:106CC000A2691143E2690243084610436146C86065
:106CD0000120A8730020F8BDFFFF00003F1FFFFF49
:106CE000F8F119FF10B500680549884207D1054839
:106CF000816B4900490881630D2000F055F810BDF3
:106D0000007C00400010024010B50068084988422D
:106D10000CD10848816BC204114381630022012118
:106D20000D2000F055F80D2000F048F810BD0000CF
:106D3000007C0040001002400068C06970470000FD
:106D400070B50224034620339C730F4C2568E6047B
:106D5000354325600468E568B6123543E56005688B
:106D6000AE6801242643AE6005682E6926432E6175
:106D70000568A96101684A6100680169042211433C
:106D800001619C73002070BD000401407047000049
:106D90000448416B012211434163816B020411439A
:106DA0008163704700100240C106C90E012088406F
:106DB000014908607047000080E100E0C106C90E8B
:106DC00001208840014908607047000000E100E0B0
:106DD00010B501F08DFA10BD02494A6882434A603D
:106DE000704700000070004002480168821511439E
:106DF000016070470070004002494A6802434A60DF
:106E000070470000007000400548016802221143ED
:106E100001600448016904221143016130BF7047D9
:106E20000070004000ED00E00A4B1A6892089200E2
:106E300002431A60084803690422134303610129CD
:106E400006D040BF20BF20BF016991430161704758
:106E500030BFF9E70070004000ED00E0F8B50446EF
:106E60000078544D800672D5524E0027403EB06BDC
:106E7000C00004D4B06BA9050843B06301274E4895
:106E80000168C90511D40168821511430160FFF73B
:106E900031FD009005E0FFF72DFD0099401A6428B0
:106EA00037D845480068C005F5D532680321090583
:106EB00060680A400140914208D08103890F03298C
:106EC00004D13168890301D50120F8BD2A69032165
:106ED00009040A4022D0084090421FD02078800642
:106EE0001CD528692A6988430121C9040A432A61FB
:106EF0002A698A432A612861C0050FD5FFF7FAFC89
:106F0000009008E0FFF7F6FC0099411A2B488142F7
:106F100001D90320F8BD28698005F3D5616888038D
:106F2000800F032805D132680005824301400A43DF
:106F30003260286903226168120411400843286105
:106F4000002F04D0B16B012000078143B16320788A
:106F5000C00705D0E868A168800880000843E860A1
:106F60002078800705D5E8680C218843E16808434C
:106F7000E8602078400706D5E86803218902884345
:106F800021690843E8602078000706D5E8680321F6
:106F90000903884361690843E8602078000606D544
:106FA000E868032189048843A1690843E860002058
:106FB000F8BD00004010024000700040881300003F
:106FC000F8B50E4605007DD053480068C007C00FD5
:106FD000B0420AD250480168490849003143016073
:106FE0000068C007C00FB04271D128784B4C8007B1
:106FF00005D5E068F0218843A9680843E060287857
:10700000C00752D06868022817D0032818D021681A
:10701000012818D08905002959DAE1688908890012
:107020000143E160FFF766FC69680746022912D058
:1070300003291CD0012926D033E021688903EAE71F
:1070400021688901E7E74907E5E7FFF753FCC11B22
:107050003348814223D8E0680007800F0228F4D12A
:1070600023E0FFF747FCC11B2D48814217D8E06899
:107070000007800F0328F4D117E0FFF73BFCC11B8A
:10708000274881420BD8E0680007800F0128F4D11F
:107090000BE0FFF72FFCC11B2148814201D90320DF
:1070A000F8BDE0680007800FF3D11B480168C907ED
:1070B000C90FB1420DD90168490849003143016047
:1070C000006800E003E0C007C00FB04201D001201B
:1070D000F8BD2878400706D5E068072109028843F3
:1070E000E9680843E0602878000707D5E0680721D1
:1070F000C90288432969C9000843E06000F036F8F6
:10710000E168084A0906090F515CC8400649086051
:107110000020FFF711FCF8BD0020024000100240E3
:1071200088130000C2A900081C010020044805497A
:107130000068C968044A4905490F515CC840704756
:107140001C01002000100240DBA90008044805498A
:107150000068C968044A8904490F515CC8407047F7
:107160001C01002000100240DBA9000810B5184ADD
:10717000D1680C20084004280BD0082810D00C2817
:1071800010D050680004410F0120C003491C884002
:1071900010BD1068C00601D50E4810BD0E4810BDC8
:1071A0000E4810BD88020E4B000F185C0902D36810
:1071B000890F491CDB0301D5084A05E01268D20695
:1071C00001D5044A00E0044A5043FDF791FF10BD89
:1071D0000010024000093D000024F40000127A0073
:1071E000D2A90008FEB505007ED0FE4CE7680C2051
:1071F000E66807400120000406402878C00747D011
:10720000082F05D00C2F0AD101200004864206D198
:10721000206880033CD568680028E5D038E001206C
:1072200069680004814203D121680143216011E0B3
:10723000052301221B0492049942216802D11143C3
:107240002160F1E7814321602168014000912068BD
:1072500090432060686800280DD0FFF74BFB00903A
:1072600005E0FFF747FB0099401A64287AD82068A8
:107270008003F6D50CE0FFF73DFB009005E0FFF73B
:1072800039FB0099401A6428F0D820688003F6D4AE
:107290002878800755D50923E868042F0DD00C2FD6
:1072A00001D1002E09D000283BD021689943014329
:1072B0002160FFF71FFB064627E02168490701D53B
:1072C000002891D061681F22120291432A6912029C
:1072D000114361602168994301432160FFF746FF34
:1072E000E16809060A0F00E079E1BF49895CC840FE
:1072F000BE4908600020FFF71FFB002872D120E084
:10730000FFF7F8FA801B0228B0D820684007F7D5AD
:1073100060681F21090288432969090208436060E7
:107320000FE02068400840002060FFF7E3FA0646BF
:1073300004E0FFF7DFFA801B022897D82068400797
:10734000F7D42878C0065FD5002F0CD0A869002894
:1073500049D02068FF21013108432060FFF7CAFAB5
:1073600006462DE0C0E02068800502D5A869002807
:10737000A7D06068072149038843296A08436060F1
:107380006068297F0002000A090608436060286AD5
:10739000410B0120C003491C8840E16809060A0F1F
:1073A0009149895CC840914908600020FFF7C4FA00
:1073B000002817D128E0FFF79DFA801B0228A3D8E8
:1073C00020688005F7D56068072149038843296A4A
:1073D000084360606068297F0002000A09060843CC
:1073E000606011E0E1E02168FF200130814321600D
:1073F000FFF780FA064604E0FFF77CFA801B0228BC
:1074000072D820688005F7D42878794E000724D5F3
:1074100068690028306910D0012108433061FFF706
:1074200069FA009005E0FFF765FA0099401A022812
:107430005AD830698007F6D50FE040084000306127
:10744000FFF758FA009005E0FFF754FA0099401A48
:10745000022849D830698007F6D42878400765D5D6
:1074600000200290A06BC00006D4A06B0121090788
:107470000843A063012002905E480168C90511D449
:107480000168821511430160FFF734FA009005E0AE
:10749000FFF730FA0099401A642825D8554800684B
:1074A000C005F5D5FF20AA680130824203D13169B9
:1074B0000143316111E001218902002A07D005232F
:1074C0001B029A4203D132690A433261EFE7326903
:1074D00082433261306988433061A86800280FD048
:1074E000FFF708FA009007E05EE0FFF703FA009963
:1074F000411A4148814257D830698005F5D50DE0E1
:10750000FFF7F8F9009006E0FFF7F4F90099411A47
:107510003948814248D830698005F5D4029800285E
:1075200004D0A06B012109078843A063686A002882
:1075300064D00C2F3ED0012636060228206805D0E4
:10754000B0432060FFF7D6F905462FE0B043206036
:10755000FFF7D0F9074604E0FFF7CCF9C01B02287B
:1075600022D820688001F7D4E96AA86AE268084353
:10757000296BFD231B049A4311430843E0602068F4
:1075800030432060FFF7B6F9054604E0FFF7B2F993
:10759000401B022808D820688001F7D52EE0FFF7AD
:1075A000A9F9401B022801D90320FEBD20688001F3
:1075B000F5D423E00128F8D0E06801210904AA6A83
:1075C000014091420BD10F218904EA6A01409142A6
:1075D00005D1032189050840296B88420ED001207E
:1075E000FEBD000000100240C2A900081C010020DE
:1075F0004010024000700040881300000020EFE7B8
:1076000070B5040007D0002625464035A662687C88
:10761000002802D005E0012070BD2E74204600F045
:107620002FF80220687420680168402291430160AD
:10763000A168606822690843E168114308436169F1
:1076400001220843A169520211400843E16908433D
:10765000216A0843A16A084321680860A0690421DF
:10766000000C0840616A0843216848602068C169CD
:1076700092009143C161666501206874002070BD6D
:1076800010B586B0044614216846FDF790FD1049F8
:107690002068884219D10F48416B8214114341631D
:1076A000C16A01221143C162C06A002110400590E5
:1076B000E0200090022001900320039002910491A9
:1076C000052069460007FFF749F806B010BD000025
:1076D0000030014000100240094910B5401E8842A8
:1076E00001D9012010BD074C60610321081F00F083
:1076F000FFFD0020A06107202061002010BD0000D8
:10770000FFFFFF0000E000E070477047F8B5026837
:107710000446D0691168936805072D0F5BD0DD071B
:10772000ED0FFF2621360E402E4367D0C60706D048
:10773000CE0504D501261662E26F3243E267870761
:1077400002220426002F06DADF0704D027683A62F7
:10775000E76F3743E767470706D5DB0704D02368A1
:107760001E62E36F1343E367020709D520220A4034
:107770002A4305D0236808221A62E36F1343E367A4
:10778000E26F002A2FD0800606D5880604D5216E28
:10779000002901D020468847E06F216889684906A2
:1077A00001D4000724D5204601F0BCFE2068816882
:1077B000490619D58168402291438160E06E002816
:1077C00012D020498163E06EFEF72EFE00280AD019
:1077D000E06E816B06E0850610D58D060ED5216E14
:1077E0001CE020468847F8BD2046FFF78EFFF8BD15
:1077F0002046FFF78AFF0020E067F8BDC50208D5E4
:107800005B0206D50120000510622046FFF77CFFD1
:10781000F8BD030605D50B0603D5616E0029E0D13E
:10782000F8BD4006FCD54806FAD51368204640212D
:107830008B431360202161670021616600F069F9C4
:10784000F8BD00008194000810B5040003D0606FFB
:10785000002802D007E0012010BD00217020015552
:10786000204600F027F82420606720680168490856
:1078700049000160204601F09FFE0128ECD0606ABB
:10788000002802D0204601F0DDFC20684168092272
:10789000D20291434160206881682A22914381602D
:1078A00020680168012211430160204601F030FD8B
:1078B00010BD0000F0B587B0064614216846FDF7FC
:1078C00076FC2C493068884251D12B48416B01220B
:1078D000920311434163C16A01221143C162C06A2C
:1078E000002510400590032040020090022003274D
:1078F00001A9A1C104200490052069460007FEF7F4
:107900002DFF1F4C1D48A560E56081C48027E56000
:10791000A7602020256160610002A0611848083C32
:10792000FEF7FCFD002801D0FEF740F9F466A662E0
:10793000144C124821461438206003206060102047
:107940000831A1C16561A561E56120462562FEF7A8
:10795000E5FD002801D0FEF729F9B46600220121D7
:107960001B20A662FFF734FA1B20FFF727FA07B0A7
:10797000F0BD00000038014000100240300002401D
:1079800078150020C0150020F8B50446806F202827
:107990004DD100290BD0002A09D00123A0681B0378
:1079A000984206D12069002803D1C80701D00120E0
:1079B000F8BD25466035287C012838D00120287480
:1079C0005820616502530026E6672220A067E06E1A
:1079D000002819D01749C162E16E17480863E16EAB
:1079E00016484863E06E13468663676D21683A4621
:1079F0002431E06EFEF7DAFD002805D01020E067A4
:107A00002E7420206067D2E72E7420680168FF2260
:107A100001321143016020688168012211438160B5
:107A2000206881684022114381600020F8BD022057
:107A3000F8BD0000DD9400081B950008959400082F
:107A400070477047FFB50446406F83B017460D4638
:107A500020285CD1002D0AD0002F08D0A168C001D9
:107A6000814207D12069002804D1E80702D0012013
:107A700007B0F0BD204660300290007C012846D05F
:107A80000298012101740020E06721206067FEF761
:107A900031FF264640360190378277820120A16867
:107AA0000003814202D12069002802D02F46002520
:107AB00011E000270FE000228021204601F090FE17
:107AC000002815D1002F15D02168387888627F1CD6
:107AD000708A401E7082708A019B00280698009070
:107AE000E9D100224021204601F07AFE002808D08A
:107AF0000320BDE728882168C005C00D8862AD1C41
:107B0000E6E720206067029900200874B0E70220B1
:107B1000AEE7704701490248C160FDE70400FA057D
:107B200000ED00E010B505242407002204212046C2
:107B3000FEF7D9FE002208212046FEF7D4FE0A20D7
:107B400002F04DF9012204212046FEF7CCFE0A2066
:107B500002F045F9002204212046FEF7C4FE10BDC4
:107B600010B505242407002204212046FEF7BBFEA1
:107B7000012208212046FEF7B6FE0A2002F02FF966
:107B8000012204212046FEF7AEFE0A2002F027F96A
:107B9000002204212046FEF7A6FE10BDF8B5002401
:107BA0000526074625463607002204213046FEF703
:107BB0009AFE0A2002F013F9012204213046FEF752
:107BC00092FE6006040E08213046FEF783FE002870
:107BD00001D0641CE4B2052002F001F96D1CEDB285
:107BE000082DE1D3002F03D0FFF79CFF2046F8BDFE
:107BF000FFF7B6FFFAE770B50526054636070022FF
:107C000004213046FEF76FFE0024E80901D001226E
:107C100000E0002208213046FEF765FE6806050EEA
:107C20000A2002F0DCF8012204213046FEF75BFE58
:107C30000A2002F0D4F8002204213046FEF753FE59
:107C40000A2002F0CCF8641CE4B2082CDDD370BD2D
:107C500010B505242407012208212046FEF743FE23
:107C6000012204212046FEF73EFE00220821204684
:107C7000FEF739FE0A2002F0B2F800220421204665
:107C8000FEF731FE10BD10B50524240700220421A3
:107C90002046FEF728FE002208212046FEF723FE9C
:107CA0000A2002F09CF8012204212046FEF71BFE68
:107CB000012208212046FEF716FE0A2002F08FF866
:107CC00010BD70B505252D07002401220821284686
:107CD000FEF709FE062002F082F801220421284660
:107CE000FEF701FE062002F07AF807E0641CE4B219
:107CF000FA2C03D9FFF7C7FF012070BD08212846E1
:107D0000FEF7E8FD0028F1D1002204212846FEF705
:107D1000EAFD002070BD0000F8B501F029FB01F07C
:107D200063FB46480068C069FEF730F84449454E99
:107D3000898F002914D044490A7801218902002A38
:107D40000AD0012A04D0022A04D0032A08D103E071
:107D5000212801D2002200E001223046FEF7C3FDB7
:107D60000121C9023046FEF7B5FD0127FF03374D5B
:107D70000024002825D036480460287A002803D142
:107D80000120287201F070FD2878632806D90022AE
:107D900008213046FEF7A7FD012205E00122082157
:107DA0003046FEF7A0FD0022052039460007FEF709
:107DB0009AFD234D274E4035A88C274F012803D02C
:107DC0001CE02C720022EAE724486946088072B65B
:107DD00080212348FDF702FF002804D002226946D3
:107DE0001F48FDF79FFF62B61EA001F0DBFDAC84CB
:107DF00002F068FD642001F0EBFFFE60688C012852
:107E000008D10F486C84048002F05CFD642001F00E
:107E1000DFFFFE60288C012806D12C8402F052FD81
:107E2000642001F0D5FFFE600548124A01889142A6
:107E300002D1C088002800D1FE60F8BDF8140020EF
:107E4000500D00200004005069000020D4000020E4
:107E5000100100200400FA0500ED00E0AAAA0000CD
:107E6000384A0008BDF8C8EBC9FDBCB6C4A3CABDFA
:107E70000D0A0000AA55000008B53721202000F0A7
:107E80006EF80321212000F06AF84021222000F042
:107E900066F80821232000F062F8AA21302000F0C3
:107EA0005EF80A48008FC1B2322000F058F8022173
:107EB000332000F054F85F21202000F050F868468D
:107EC00000F006F80A2001F08AFF08BD500D0020DE
:107ED00010B501460F2000F021F8002800D0012045
:107EE00010BD10B50446FFF7B3FE3220FFF783FE46
:107EF000FFF7E7FEE0B2FFF77EFEFFF7E2FEFFF7D7
:107F0000A7FE3320FFF777FEFFF7DBFE0020FFF729
:107F100045FE0446FFF7B7FE204610BD10B50C46DF
:107F2000FFF7DFFF2070012010BD70B50D4604463D
:107F3000FFF78EFE3220FFF75EFEFFF7C2FEE0B2D3
:107F4000FFF759FEFFF7BDFE2846FFF754FEFFF787
:107F5000B8FEFFF798FE0A2001F041FF70BD10B592
:107F6000FFF7E3FF012010BD10B50248FEF704FE45
:107F700010BD000070140020FEB50446002572B646
:107F80000068394A831804D13849CD68032189042F
:107F90000D4081680191C168009141698669002B9B
:107FA00008D132484038836AC7043B438362836AFE
:107FB000BB4383620846304348D02B482368C34202
:107FC00005D12A48C368032292049343C360002961
:107FD00017D02068026901231A43026120684161B9
:107FE000FEF788FC0746FEF785FC2168C01B096880
:107FF000090703D47D21C9008842F4D921680820EB
:108000004860002E17D020680169012211430161E8
:1080100020688661FEF76EFC7D270646FF00FEF7AE
:1080200069FC2168801B0968C90601D4B842F6D9E9
:108030002168102048600C482168C14206D10B48D5
:10804000C1680322920491432943C16020680169F9
:1080500049084900016121680198886021680098F9
:10806000C86062B6FEBD00000084FFBF4010024041
:108070001CB5002116480091144A01910260C163A9
:10808000120542608160072282630122026102467A
:10809000C16020321170FF235170C233436281628C
:1080A000117301638161042241634261C161FEF782
:1080B00021F8084800908013019069460448FDF7B4
:1080C000C9FF00210248FDF76FFF1CBD00240140DD
:1080D000141400200200000408B50848016B0122B6
:1080E00011430163006B01211040009000220A201F
:1080F000FEF76EFE0A20FEF761FE08BD001002408A
:10810000F0B587B014216846FDF751F84C48C26AB3
:1081100004210A43C262C26A0A400592C16A8027EA
:108120003943C162C16A39400591C16A01252943B9
:10813000C162C16A29400591C16A02263143C16208
:10814000C06A2A463040059005201C210007FEF732
:10815000CAFB01223B493C48FEF7C5FB00223B49D4
:108160003948FEF7C0FB91210520002209020007D3
:10817000FEF7B9FB364801900024052069460095BA
:1081800002940007FEF7EAFA0320019005206946F1
:10819000009602940007FEF7E1FA0C2000901120EF
:1081A0000190032003900520029469460007FEF722
:1081B000D5FA102000900520694603960195029497
:1081C0000007FEF7CBFA1120019002946946009552
:1081D00003941D48FEF7C2FA1E48019069460096B6
:1081E00002951948FEF7BAFA1B48009002946946B6
:1081F000019503941448FEF7B1FAE8026A4651C2A9
:1082000069461148FEF7AAFA912000020090052065
:1082100002946946019503940007FEF79FFA6946A8
:108220000948009702950194FEF798FA002201216F
:108230000520FEF7CDFD0520FEF7C0FD07B0F0BD1F
:108240000010024001060000000400500830000049
:1082500000001110000021100836000010B50F4C6E
:108260000D482060FF20053060600020A060E060C5
:1082700020616061E0610121206249026062A161C8
:10828000A0620720E0622046FFF7BAF92068016883
:1082900040221143016010BD00300140A0140020B5
:1082A00000B585B014216846FCF781FF0E480D49E2
:1082B0000160E1214902416000218160C1600161EA
:1082C00081610C22C1614261016230214162012160
:1082D000090381634900C163FFF7B6FA01F0BEFAF2
:1082E00005B000BD00380140F814002070470000C0
:1082F0008307FF22DB0E9A408907090E9940002868
:108300000BDA0007000F0838830808489B0018188C
:10831000C36993430B43C3617047830804489B00C0
:108320001B181868904308431860704700ED00E080
:1083300000E400E0BFF34F8F04490348C860BFF377
:108340004F8F00BFFDE700000400FA0500ED00E0DC
:10835000F0B587B00A2002F02BF87D20C00002F0B3
:1083600041F8FA4C0025A570607B0C2801D30B2046
:1083700060730122052051020007FEF7B4FA0026BF
:10838000F348E670F34D00782871F349A079097835
:1083900040000843E17C89000843E871A06AE87066
:1083A000401CA06260792946A8744200B431084696
:1083B000A138FCF7E3FE06206872E8480022007846
:1083C000A872A07E287328461338217F0175617F2B
:1083D0004175607929464000153002F0D3F8607984
:1083E00000214000153002F0DFF8022002F030F8E2
:1083F000EE71E673A67201202073E672D848FEF78C
:108400009BFC20840546E6706079FDF737F9D54A74
:10841000D54BFDF72DF801F077FC012300229B07D7
:10842000FCF774FFFDF770F90006C00C401980B22C
:108430000121C9036084884201D3401A6084CB487B
:1084400060632079401C2071C548FEF775FCE0830D
:10845000C0480C300646423640300390ABE1C0487D
:10846000FEF76AFC2546E083C14F0BE0BC48FEF7EF
:1084700063FC80B2E8836A8C904203D3BD495118F3
:10848000884206D300210F2001F012FF3842E86233
:10849000ECD0E86A411C20D040047DD58122D20175
:1084A00000210F2002F043F87D20C00001F09AFF68
:1084B000002001F04CFF0021102001F0F9FE4106E0
:1084C000A448490E00225030696401F027FFA148FA
:1084D0005030417A0729C1D101E0FFF72BFF02227A
:1084E000A549401DFCF76EFE0028B7D102F0ADF89B
:1084F0006965286502F096F8E965A865E878694637
:10850000401CE87093484D3002790A7040794870F9
:1085100008880090A98B884275D1984D308A2880B0
:108520000398808A20838E48FEF706FCE08301F0E2
:10853000D1FDFF23A06D5B04E16D0022C018514105
:108540000906070A0F4378084000010E0002616621
:1085500020668048636D0A30226D02F04BF8607926
:10856000E36D81007B48A26D0818163002F042F8D6
:108570007848636E1230226E02F03CF8754808218C
:10858000417260790022800072491C3001F0FAFFCC
:1085900060798000002100E000E11C3002F004F866
:1085A000384601F0FEFE012001F052FF2072022148
:1085B0007348FEF78FF9002826D000216648634AE9
:1085C0000170B0891086F1895186624B226B50335D
:1085D0006263DA7C1607360F032E00D06674120928
:1085E0000027A27401262771584BA6729886D98657
:1085F000002A18D0574802225F495530FCF7E2FDA7
:10860000002803D00FE075E00121D7E75148E67359
:10861000C671606C4F491638C2B266310846227482
:10862000D230FCF7ABFDE672208B5649FF30C330E9
:1086300080B2208388420BD9494240182083288881
:108640007D21401C80B2C9002880884200D32F8041
:108650002D887D20C000218B68434018A0630690C0
:108660004948302107784948A77300884843FCF7F8
:10867000EAFF009028460A214843FCF7E4FF0099EE
:10868000FCF706FE7F21C905FCF7A9FDFDF704F8FC
:1086900080B23D497F1E0880B84200D1E672A584B1
:1086A0001420205EFCF7D6FF06460F46E08BFCF751
:1086B000E5FF374A374BFCF7DBFE05460591069888
:1086C000FCF7C8FF2A46059BFCF7C4FE32463B4632
:1086D000FCF71CFEFCF7F4FFE063608B00F094FCF9
:1086E000207A002870D100210F2001F0E1FD000662
:1086F000F9D569E0FDF732FB274A032111541349EC
:10870000B28987000A862448F2894A866038391877
:108710000398008B08802049286B3039C8510D48D8
:10872000EB6D38181630AA6D01F064FF1A48296BFA
:108730006038C05988423EDD00283CD000293ADD2F
:108740000098A8830220287035E00000580000201F
:10875000D4000020C41100200C010020E6000020FD
:1087600070140020B81E85EB51B8CE3FA0860100E2
:1087700000D02724983A0000F400002008010020CF
:1087800000040050E7030000EC000020F00000208F
:10879000F853E3A59B843E40F01200203A460021A6
:1087A0000F2001F0C4FE6879E978401C814202D0B4
:1087B000002001F0CCFDE08B618C884200D24EE6B7
:1087C0001B4A89188842FAD801F084FC194A002112
:1087D0000F2001F0ACFE18480A2100884843217997
:1087E000884201D200202070E07B002805D0134988
:1087F00008784B788A7802280ED00E4A0021803201
:108800000F2001F094FE01210520002249020007FB
:10881000FEF769F807B0F0BD0948C91CC018FCF79D
:10882000ADFC02F04FF8642001F0D2FA55E60000EA
:10883000983A000000D02724E6000020FC12002017
:10884000500D002070470000F0B58DB0B448019085
:108850000020C0430A9000260A2001F0A9FD7D20D7
:10886000C00001F0BFFD0020AE4C0546A070AE4F29
:10887000AE480B90AD480022C238857301461420E3
:1088800001F080FE0021142001F08EFE022001F094
:10889000DFFD00210F2001F00BFD3842E062F8D02F
:1088A000E06A411C18D040047ED58122D20100210B
:1088B0000F2001F03CFE0021102001F0F9FC4106E0
:1088C0009A48490E0022801C01F028FD9748801C20
:1088D000417A022902D007E1FFF72CFD93480222DA
:1088E0009349C01DFCF76EFC0028F4D101F0ADFEE9
:1088F0006165206501F096FEE165A065002E22D13C
:108900000B988C49008A088088480126801E808A3E
:1089100020838948FEF710FAE083208B8749FF30D7
:10892000C33080B2208388420DD949424018814922
:1089300020830888814A401C80B20B320880904214
:1089400001D3002008800B9968468A890280C98972
:10895000418076490422C91C0846A238FCF70EFC67
:10896000FF22A16D5204E06D0023891858410006D2
:10897000090A01430846029101F013FD02994808D3
:108980004000010E0002616620666848636D9638FB
:10899000226D01F02FFE6548E36D9238A26D01F063
:1089A00029FE62488E3800E0A0E0636E226E01F07E
:1089B00021FE5E490022A0393C2001F0E3FD0021A8
:1089C0003C2001F0F1FD012001F042FD2072A07871
:1089D0000121401CA0700520C9030007FDF7D2F952
:1089E00054487D220088D200014602905043228BD9
:1089F0000A398018A0630C9051480078A073049045
:108A000008B2E084002803DA7D21C9004018E08420
:108A10004C48302100884843FCF715FE059026207D
:108A2000205EFCF705FE0599FCF732FC7F21C905A5
:108A3000FCF7D5FBFCF730FE414980B20880049971
:108A4000491E884201D10120E0720298A0841420BE
:108A5000205EFCF7FFFD05910690E08BFCF70EFE13
:108A6000394A3A4BFCF704FD079104900C98FCF747
:108A7000F1FD079B049AFCF7EDFC059B069AFCF7B9
:108A800045FCFCF71DFEE063608B00F0BDFA009929
:108A90000198814210DA00290ED024490422C91C11
:108AA0000AA8FCF76BFB0220207029480A210078F5
:108AB0004843607200980190207A002805D1002177
:108AC0000F2001F0F5FB0006F9D5802200210F20D0
:108AD00001F02DFD00206D1CEDB26070032D00D261
:108AE000C8E6002E08D017E00120F4E7194A00215B
:108AF0000F2001F01CFDF7E7618B1748002902D019
:108B00000288914201D90188618388B21349401ECD
:108B100009884843124908800A98A0830DB0F0BD27
:108B20003F420F005800002000D0272412120020DE
:108B3000F40000200801002070140020E70300006A
:108B4000EC000020F0000020F853E3A59B843E4099
:108B5000E600002000902724E2000020E000002032
:108B6000DE000020F8B53A493848086001F04AFEB6
:108B7000394C38486080204640300079374D000637
:108B8000000EA87003D0E08800280AD00BE07D20FA
:108B9000C000E0800120E0870A2060870020A087D5
:108BA00001E06420E080208F0A2801D9022020877C
:108BB000E08E3C2801D93C20E086294980B208702B
:108BC000E08FA871A08FE871A07A2871A68805218E
:108BD0002E62A981E7883846FCF78AFAE8810146C7
:108BE0003046FCF785FA8800081886B27D20C00060
:108BF0006E817043FCF742FD1A4A1B4BFCF7A0FC48
:108C0000FCF782FD28827D20AE823946C000FCF749
:108C10006FFA68820146C820FCF76AFAA88301202F
:108C20002883FDF7B3F8E8822A8A10491048FEF736
:108C300087F810A0296A00F0B5FEE18811A000F0C5
:108C4000B1FE218914A000F0ADFEF8BD9598000892
:108C5000500000200E020000500D0020D400002023
:108C600000000020F853E3A59B843E40FF7F0000F6
:108C700070140020B1EAC7A949443A202564202E87
:108C80000D0A0000CDA8D1B6BCE4B8F43A202564A2
:108C9000206D732E0D0A0000B5A5B4CECDA8D1B6B7
:108CA000BBF9D5BECAFDC1BF3A202564B8F62E0D6A
:108CB0000A000000F0B5904D85B0012028808F4F4C
:108CC000C8208F4C3880E079401CE071C00706D086
:108CD000608B411E6183022801D2C8206083608BB3
:108CE00000F092F90A2001F063FB7D20C00001F042
:108CF00079FB02218348FDF7EDFD002838D00020E4
:108D0000814980000978824E490008437F490978EB
:108D10000843B072102070727E48C1887D20C00068
:108D2000FCF7E6F970737C487A490078B0733046F6
:108D30000B308A780270C9784170411C7548203028
:108D4000027ECA70407E087172482230027E4A71EB
:108D5000407E887100220C39152001F013FC00219F
:108D6000152001F021FC022001F072FB6B4E03E0A4
:108D70000120C5E7FEF7D0FF00210F2001F098FA8F
:108D80003042E062F6D0E06A411C7DD040047CD5E0
:108D90008122D20100210F2001F0C9FB0021102007
:108DA00001F086FA41065A48490E002250306164AB
:108DB00001F0B4FA564E5036707A112865D102226D
:108DC0005749701DFCF7FEF900285ED1F01E0279AC
:108DD00069460A7040794870B17A2980C820FCF74A
:108DE00087F93880307B60834E4DB01E008A288022
:108DF000301F808A20834C48FDF79EFF80B2E083BD
:108E00000390208B4949FF30C33080B220838842D1
:108E10000CD949424018208328884449401C80B21C
:108E20000B312880884201D3002028802D887D20A6
:108E3000C000218B68434018A06302903C4806782C
:108E400028460A3800B2A673E084002803DA7D21A0
:108E5000C9004018E084388830214843FCF7F3FB10
:108E600007462620205EFCF7E3FB3946FCF710FAA4
:108E70007F21C905FCF7B3F9FCF70EFC81B22C4841
:108E8000761E0180B14201E033E030E001D10120E3
:108E9000E072A5841420205EFCF7DCFB07460191FC
:108EA0000398FCF7EBFB234A234BFCF7E1FA05465A
:108EB0000E460298FCF7CEFB2A463346FCF7CAFA68
:108EC0003A46019BFCF722FAFCF7FAFBE06368469E
:108ED0000088A0830E480E495030807C60714200AB
:108EE000633108465130FCF749F90320207005B082
:108EF000F0BDFFF71FFA0000E6000020F0000020A0
:108F00005800002000040050DA000020DB000020A0
:108F1000C4110020500D00200000002000D02724A4
:108F2000F40000200801002070140020E703000076
:108F3000EC000020F853E3A59B843E4070B586B05A
:108F400014216846FCF733F901250F4EED0300228A
:108F500029463046FDF7C7FC012000240190029409
:108F60006946009503943046FDF7F8FB0320019015
:108F700002946946009503943046FDF7EFFB02200A
:108F800000F026FF06B070BD0004005070470000DE
:108F9000F8B5044600206A461080194D55222A7003
:108FA000AA226A700322AA70661DEE702A71697186
:108FB000144A49008918AC712246E81DFCF7DEF816
:108FC000002007E029186A468978128889186A46BD
:108FD0001180401CB042F5DB611DA81CFCF72AFD86
:108FE00001466846018029190078C87168464078B2
:108FF000087221460931024800F0ACFAF8BD0000C1
:10900000B0130020500D002010B51D481D4C007DF0
:109010001D4960700880218B628A914201D3891AB0
:10902000218389B2A28B0B4653431B1863831329F8
:1090300002D14A4310186083608B30214843642179
:10904000643048431149E0620968401A10494018E9
:10905000A062FCF7FFFA0F4A0F4BFCF771FAFCF71E
:109060002FFB0E496062884202DD4A42801860622E
:10907000002801DA4018606209490968486110BD9A
:10908000500D0020D4000020720000209400002029
:10909000F0D8FFFFF853E3A59B843E40FF7F00001C
:1090A00070140020034A1168382389B299430143A0
:1090B000116070470030014010B5FDF721FC10BD74
:1090C00010B59AB034216846FCF771F814210DA848
:1090D000FCF76DF81C2112A8FCF769F81B48016821
:1090E0000324E402A143C21489180160FDF77CFE49
:1090F00017480169A143016106200090FF2001305B
:109100000290012003901020049002200990400456
:109110000B90000100240C900A946846FEF762F858
:109120000F200D9003200E900F94109401211194A4
:109130000DA8FDF745FF81201290032080041890B0
:10914000149412A8FDF78AFE1AB010BD00700040FA
:109150004010024010480168821511430160C16847
:109160000E4A1140C16001680D4A114001608168DA
:10917000490849008160016801229204914301601D
:10918000C168FD2212049143C160002101610649BA
:109190000448886070470000001002400C40FF88BF
:1091A000F6FFF6FE0050000800ED00E070B501F09B
:1091B00093F8224C224DA06402E001F08DF8A064E7
:1091C000A842FAD1207801260525F6032D070028AC
:1091D00006D001280CD0022817D003282BD128E074
:1091E000012231462846FDF77EFBFFF763FD06E0CE
:1091F000012231462846FDF776FBFFF725FB0022CA
:1092000031462846FDF76FFB15E0607A0122401ECB
:10921000607231462846FDF766FBFCF7D3FD00225D
:1092200031462846FDF75FFB607A002803D12070A5
:1092300001E0FFF78DF800F035FF70BD5800002009
:109240003001CADE10B5818CC90707D001684A68B1
:1092500001235B049A43836A1A434A60818C89071D
:1092600007D501684A6801231B049A43C36A1A435D
:109270004A60818C490707D501684A6801239B042D
:109280009A43036B1A434A60818C090707D501682A
:109290004A680123DB039A43436B1A434A60818C7B
:1092A000C90607D50268916801231B039943836BA4
:1092B00019439160818C890607D501688A6801236A
:1092C0005B039A43C36B1A438A60818C490612D5AB
:1092D00003685A6801210905046C8A4322435A60D5
:1092E000026C8A4207D10268516803235B059943E7
:1092F000436C19435160818C090607D501684A689F
:109300000123DB04806C9A4302434A6010BD0000D5
:10931000F8B500260446C667FDF7ECFA0546206856
:109320000068124F000709D501212B46002249058C
:109330002046009700F054FA00280DD120680068FC
:1093400040070BD501212B460022890520460097B6
:1093500000F046FA002801D00320F8BD2020606705
:10936000A067603426740020F8BD0000FFFFFF01F5
:10937000F8B5184CC826E078002829D16079002873
:1093800026D101206071144D686B002700281ED083
:10939000686BC821081A15E01048E168405C6169F3
:1093A00088470F480A21008848430E490880E06832
:1093B000401CE060E068C82800DBE760696BC820FB
:1093C000401A761EE168814201D0002EE4DC67710C
:1093D000F8BD00003C00002000000240880C002086
:1093E000E6000020F200002070B5224CE078002852
:1093F0003FD1207900283CD1012020711E4EF16917
:1094000000250906002933DA2156625791420AD114
:10941000F06940062CD5A079002829D0A5712089B3
:10942000401C208124E0A179002903D1A0710A20E9
:1094300000F0D5FC00202056CC2148430F494218AB
:10944000206912181279B262401C00222061A256D3
:10945000CC235A43895881420ADC25612078401C7C
:10946000207020780E2800D12570A078401CA070B4
:10947000257170BD3C0000200038014060010020D3
:1094800010B5806A0022014640314A834A82FEF7C5
:109490003CF910BD70B5846A606FA56F216889685A
:1094A00000260906002906DA212804D15220065395
:1094B000204600F047F820688068400606D5222D37
:1094C00004D15A200653204600F02CF8E06F1021FA
:1094D0000843E0672046FEF718F970BD10B5014655
:1094E0000968806A0968890614D400225A210A5240
:1094F00001680A68FF2301339A430A6001688A6899
:10950000520852008A6001688A6840239A438A6040
:1095100020218167FEF794FA10BD10B5806AFEF72E
:1095200090FA10BD01680A68FF2321339A430A604C
:1095300001688A68520852008A60202181670021F0
:109540000166704701680A68C0239A430A602021B7
:109550004167704770B5164CE278002A0CD1227929
:10956000002A09D10122E2700025C82903DC022269
:10957000A256002A01DCE57070BD0123E356CC221F
:1095800053430C4AD1500123E356CC2673439B1816
:109590000A460146181DFBF7F1FD6078401C60701B
:1095A00060780E2800D16570A078401EA070E2E7B8
:1095B0003C00002060010020F8B504462669A2683E
:1095C000E76932436669102000253E432368324331
:1095D00078491E68784F3E4016431E6023685A68DB
:1095E00003263603B243E66832435A602368A26911
:1095F0008B4201D0266A32439E680B273F02BE434E
:1096000016439E606D4E23686D4AB3420CD1D268FA
:109610009207920F06D0012A38D0022A34D0032AAA
:1096200020D11EE001201DE0664EB3420AD1D2686F
:109630000C26324026D0042A28D0082A24D00C2A0E
:1096400010D10EE08B420DD1D66803229202164053
:1096500018D001229202B61A18D0B61A14D0964227
:1096600000D10820564A0126403A574FF6038B4254
:1096700036D100280CD002280DD0042812D008289A
:109680001FD11CE00020EDE70220EBE70420E9E712
:10969000FDF74CFD08E01068C00601D5384605E02E
:1096A0004A4803E0FDF762FD002873D0626851006C
:1096B0005118814205D81103814202D303E030469C
:1096C000F4E7012566E0010E060250080023301879
:1096D0005941FBF723FD03210902411A3C4A55E099
:1096E000E169B14232D1030000F083F909070A0DA4
:1096F00006250606062B0600E3E7FDF717FD1CE02E
:10970000FDF724FD19E010686168C00602D548081D
:10971000304A01E0304A48088018FBF7E9FC80B283
:1097200001462E4A10399142CBD8511C0140000706
:10973000400F08432CE0FDF719FD616840004A081E
:10974000EAE76168012248081204E5E7030000F037
:1097500050F909070A0D06260606062C0600B0E792
:10976000FDF7E4FC1DE0FDF7F1FC1AE0106861680C
:10977000C00602D54808C01902E014484A0810186B
:10978000FBF7B6FC80B20146144A1039914298D8D2
:109790002168C8600020206660662846F8BDFDF795
:1097A000E5FC61684A088018EAE7616848088019A2
:1097B000E6E7000000480040F369FFEF0038014091
:1097C000401002400044004000093D000024F40025
:1097D000FFFC0F0000127A000048E801EFFF0000D4
:1097E000FFB581B017460E4604460A9D09E0681C85
:1097F00007D0FDF77FF80499401AA8420CD8002D35
:109800000AD02068C1693046884318D00020B84289
:10981000EDD0002005B0F0BD20680168FF22A13224
:1098200091430160206881684908490081602020D7
:109830006067A0670020603420740320EAE70120FD
:10984000E5E7000010B504491020096808620248E5
:10985000FDF75CFF10BD0000F814002001490D2049
:10986000887070473C00002010B507480A22418AE2
:109870005143C183FEF730FCFEF712FDC8220349B5
:109880000348FEF781F810BDD4000020880C0020AA
:10989000F8140020F8B53E4C002321783D4A1D46BF
:1098A000082910D0072947D0062950D0052952D0C1
:1098B000042953D0032954D0002956D0012958D067
:1098C00002295AD05BE0A17800264A1F04E0314FFC
:1098D000BF5DFB189BB2761C9642F8DB6679277950
:1098E0009A195118E3786278C9188918C91940186B
:1098F000C0430006000E1AD1012E14D0022E16D13C
:1099000025482449C018FBF739FC00F0DBFF642030
:1099100000F05EFABFF34F8F21492048C860BFF3C3
:109920004F8F00BFFDE759081046FFF731FB257048
:10993000E570A570A571F8BDA1795054491CC8B255
:10994000A071A178491F8842F5D1082001E060701C
:1099500007202070F8BDE0700620FAE7607105204E
:10996000F7E7A070E5700420F3E7552807D1012040
:10997000EFE7AA2803D10220EBE7032803D02570E4
:10998000E570A570F8BD032020702071F8BD0000BF
:10999000CB0000204C130020500D00200400FA05DD
:1099A00000ED00E00FB410B503A9044B044A02987F
:1099B00000F002F910BC08BC04B018470DA600085E
:1099C000200100202021020C01D010211046020AA3
:1099D00001D010460839020901D01046091F82083B
:1099E00001D01046891E420801D0881E7047081A0F
:1099F000704730B47446641E2578641CAB4200D2B4
:109A00001D46635D5B00E31830BC184702E008C8E0
:109A1000121F08C1002AFAD170477047002001E0E8
:109A200001C1121F002AFBD1704708B5002168460A
:109A300001706B46012202212C2000F087FD0221DB
:109A4000684601706B4601222C2000F07FFD08BDA6
:109A500038B504466D20694608706B4601220749F7
:109A60002E2000F073FD0649002C01D0054A00E0CD
:109A7000054A2E2000F050FD38BD00000608000009
:109A800006180000070600000716000038B5044657
:109A90006B4602220021362000F024FCB321230073
:109AA000FFF7A7FF0E0F08153A3A3A3A1C273A3A41
:109AB0002F34483A00216846017040784108490037
:109AC00014E06946087880088000401C04E069467C
:109AD000087880088000801C08701DE068460278C5
:109AE0000A40483202704178802001436846417044
:109AF00012E0684602780A40027040784106490E3A
:109B0000F4E7694648780221084303E0694648784B
:109B1000FD210840694648706B460122002136202D
:109B200000F014FD012200AB11463620013300F095
:109B30000DFD38BD69460878CF21084069462030C0
:109B4000CAE708B5032168464170012101706B46E0
:109B500002220021362000F0F9FC0122D203062166
:109B60002D2000F0D9FC012000F032F90120FFF790
:109B70008DFF08BD08B5020A69464A7008706B4639
:109B8000022204212D2000F0E1FC03206946087028
:109B90006B46012206212D2000F0D8FC00206946EA
:109BA00008706B46012206212D2000F0CFFC0A210F
:109BB0002D2000F07DFB08BDFFB58DB004460025CB
:109BC00006E025280AD0109A0F999047641C6D1C56
:109BD00020780028F5D1284611B0F0BD00270121DA
:109BE000484A009700E00743641C23780846203B5E
:109BF00098401042F7D120782E2817D1042007432F
:109C00006078641C2A280CD10E98641C02C800914C
:109C10000E900BE000990A22514330394018641C21
:109C200000902078014630390929F3D9207800289E
:109C3000D1D0642808D0692806D075281ED0109A83
:109C40000F9990476D1C5BE00A200E99019001C9A5
:109C50000E91002802DA40422D2102E0390504D598
:109C60002B216A461172012103E0F90704D020215B
:109C7000F7E70BAE0B910DE00021FAE70A200E99F1
:109C8000019001C90E91F7E70199FBF731FA3031E4
:109C9000761E31700028F7D103A8801B2030019078
:109CA000780701D5009801E00120009001998842D1
:109CB00001DD401A00E000200027009006E002A825
:109CC000109AC05D0F9990476D1C7F1C0B988742BE
:109CD000F5DB04E0109A30200F9990476D1C009935
:109CE000481E00900029F5DC05E03078109A761CBB
:109CF0000F9990476D1C0199481E01900029F4DCD2
:109D0000641C65E709280100F8B54A002B4B520D89
:109D1000D6182B4A0C460546142E2BDA002E12DAE2
:109D2000284BFBF7F3FA00221346FBF719FE40D24B
:109D3000002C03DA0124E40700253AE020462843FA
:109D400037D0214C14E0214F0B46F7403B402B43CA
:109D500031D01C4BFBF7DAFA00221346FBF700FE6A
:109D600027D2002C03DD01200005F0400419BC437C
:109D700000251EE0332E1EDC33460027143BFF4334
:109D8000DF40384217D00F4BFBF76AFB0022134627
:109D9000FBF7E6FD0DD2002C0ADD142E0CD034208A
:109DA000811B012088404019A84200D2641C05464E
:109DB000BD4321462846F8BD641CF9E701FCFFFFBE
:109DC0009C7500883CE4377E0000F03FFFFF0F00E9
:109DD0007D2110B5C900484300F001F810BD0021F5
:109DE00040E000BF00BF00BF00BF00BF00BF00BF1A
:109DF00000BF00BF00BF00BF00BF00BF00BF00BF6B
:109E000000BF00BF00BF00BF00BF00BF00BF00BF5A
:109E100000BF00BF00BF00BF00BF00BF00BF00BF4A
:109E200000BF00BF00BF00BF00BF00BF00BF00BF3A
:109E300000BF00BF00BF00BF00BF00BF00BF00BF2A
:109E400000BF00BF00BF00BF00BF00BF00BF00BF1A
:109E500000BF00BF00BF00BF00BF00BF00BF00BF0A
:109E600000BF491C8142BCD370470000FEB50446C8
:109E70000020019000906079734940000E5A61788B
:109E80002578491E7148CFB20163042D77D0072D84
:109E900075D000210291217801736C49E379012288
:109EA00092058969002B6CD0914381616748217AC2
:109EB0004173217A82698907890B0A4382610021F3
:109EC000042000F034FB324661492E2000F024FBD0
:109ED0003846FFF7BDFD5F4E0522705D81004018DA
:109EE0005D49431807212B2000F030FB5B490298A5
:109EF00001220B180B21282000F028FB705D584927
:109F000080000A580C21282000F011FBE079554907
:109F100080004018A1794900425A0221272000F010
:109F2000FBFA51487E00825B0421272000F0F4FAFE
:109F3000E079002829D0A07804282CD02820694670
:109F4000087220220621272000F0E6FA02AB012247
:109F50002621272000F0FAFA444938014018E17818
:109F6000890042580821272000F0E1FAA17A601CFC
:109F7000627A0902114313D016E000E001E00121EA
:109F800088E71143F608816190E7642206212720C3
:109F900000F0C2FAE0E71020694608720246D1E7F5
:109FA00033490172090A4172417A007A0A02024376
:109FB0002021272000F0B0FA2E4F0C2123203A68F0
:109FC00000F0B5FAF01982880421232000F0A4FAE9
:109FD000A07900280BD0E0792749012243180021FD
:109FE000212000F0B3FA03200190012000902A07FD
:109FF000120F10010243607800218007000B02431A
:10A000000198000502430098400402432079C006ED
:10A01000400902436079C00602431F2000F087FA1E
:10A02000A07861780123084302040848DB03026139
:10A03000E179490319430A4302610021082000F035
:10A0400076FA0020FEBD000090A90008240100203F
:10A050000428000038A900080C0000202A00002075
:10A0600040A9000860A900086CA9000870A90008B0
:10A070004110000058A900082C00002038B50C46FB
:10A0800007498A8B002102432C2000F045FA6846DC
:10A0900004706B46012206212C2000F057FA38BDCF
:10A0A0002401002010B5FFF7C0FC10BD10B5044618
:10A0B0000421362000F0FCF80121C902002C01D057
:10A0C000084300E0884302460421362000F02FFABE
:10A0D00010BD000038B540206946087000210E20F0
:10A0E00000F0E6F80446002211460E2000F01FFAA8
:10A0F0006B46012200210D2000F028FA074A0021BA
:10A100000F2000F014FA00F0EDF9224600210E2095
:10A1100000F00DFA02480021017338BDF8FF272432
:10A1200044010020FEB50546042069460870514CE4
:10A130000020607521462031206348710873A08398
:10A140006063A06300F0C8F84B4E206002E000F0AE
:10A15000C3F82060B042FAD10020FFF797FC00F06E
:10A16000BBF8464E20603078242801D9243806E018
:10A170000621FAF7BDFF0622101A40010843020625
:10A1800001040A4301020A430243B26070600021E5
:10A190001E2000F0CCF900F09FF820606B460122F1
:10A1A0000021242000F0D2F91E20FFF7E3FC86B244
:10A1B000300AA0730420FFF7DDFC074600F08CF89E
:10A1C00020603806000E0DD002206946087101ABF0
:10A1D000012212212D2000F0B9F9A08B01210903E1
:10A1E0000843A08300F078F820600620FFF7C2FC47
:10A1F00060600720FFF7BEFCA060F006C00E20756F
:10A2000001D110202075C0B200F0DCF9E80707D0BA
:10A21000FFF797FCA08B0121C9020843A0830AE045
:10A220000521362000F02EF8154908400246052188
:10A23000362000F071F90120FFF728FC00210420EE
:10A2400000F036F8A0610021262000F031F8152139
:10A250008903084302460021262000F068F9002205
:10A260002621362000F058F900F036F82060002052
:10A27000FEBD0000240100203001CADE00000020E5
:10A28000FFFD000038B5094C89B280B26B4602224E
:10A2900000F028F8002806D1684640780102684698
:10A2A0000078081884B2204638BD0000FFFF000087
:10A2B00038B50024E44389B280B26B46042200F032
:10A2C00011F8002806D103216846435C2202D41805
:10A2D000491EFAD5204638BD10B500210846FFF7C3
:10A2E000E7FF10BD38B5002909D0402420436C4653
:10A2F0002070C8B27F2906D8607002200AE0694643
:10A300000870012006E0802420436C466070C80974
:10A31000A0700320694600F0AFFA38BD10B51446AE
:10A3200003460A4621461120FFF7DCFF10BD10B599
:10A330000346052200211520FFF7D4FF10BD10B5FC
:10A340000346052200211720FFF7CCFF10BD38B5CA
:10A35000054600206946087000F0C4F8FF24013467
:10A360002246002D01D00322120200210D2000F010
:10A37000D3F8002D13D06B46012203210F20FFF7E5
:10A38000B1FF68460078000709D5FFF7A3FE224613
:10A3900000210D2000F0C0F80020C04338BD00208F
:10A3A00038BD10B5024601210A2000F0C0F810BDEA
:10A3B00010B5044600211A20FFF77AFF000D220392
:10A3C0000005120B024300211A2000F0B0F810BD66
:10A3D00010B5024602492E2000F09EF810BD000084
:10A3E00004180000F8B505466B460122032104203D
:10A3F000FFF778FF0126114C3607002D0DD02A46B5
:10A4000000210C2000F088F86946087810210843E4
:10A4100069460870A069304307E069460878EF2173
:10A42000084069460870A069B0430B46A06101224C
:10A430000321042000F08AF8F8BD00002401002068
:10A4400010B502460021182000F066F810BD00008B
:10A45000F8B50746002568460570B807204C2E461B
:10A4600000280ADA8020694608706B460122002124
:10A470000D2000F06BF801202073F807694608787A
:10A4800021D006210843694608706B46012200214D
:10A490000D2000F05BF803210F20FFF7F3FE812170
:10A4A000C900084219D04020694608706B46012255
:10A4B00000210D2000F04AF80020FFF7F7FD0025ED
:10A4C0002673ED4309E002210843694608706B4694
:10A4D000012200210D2000F039F82846F8BD0000C7
:10A4E000440100201CB56B46012203210F20FFF719
:10A4F000F9FE684600784022C1091040C9014000B9
:10A50000814208D0012069460871024601AB03214F
:10A510000D2000F01BF81CBD08B56B461A70120A1E
:10A520005A7089B280B2022200F010F808BD38B526
:10A5300000236C46E254120A5B1C042BFADB89B23E
:10A5400080B22346042200F001F838BD38B58024DB
:10A55000002909D0C02528436D462870C8B27F293C
:10A5600007D86870022009E020436946087001207E
:10A5700004E020436870C809A8700320694600F011
:10A58000B7F938BD10B51446012312189B029A4240
:10A5900002D90020C04310BD0B46821E214609206F
:10A5A000FFF7D4FF002010BD10B5054A89051269D8
:10A5B00001430A4300210820FFF7B9FF002010BD26
:10A5C0002401002038B504466B4601220E212B20C1
:10A5D000FFF788FE68460078E10640094001C90E91
:10A5E0000143684601706B4601220E212B20FFF7C4
:10A5F000ADFF38BD10B5002142541C06120A22439B
:10A600001B0A491C0429F7DB10BD000013B5012308
:10A610001A4669460248FDF715FA00981CBD00006D
:10A62000F81400207CB5002425466846FFF77FFE1D
:10A6300004206946220E2D02154322020C5C1443AD
:10A64000401EF7D5204629467CBD7CB50024254612
:10A650006846FFF774FE04206946220E2D0215435A
:10A6600022020C5C1443401EF7D5204629467CBDCF
:10A67000FCF74EF9FEF724FDFDF742FD3C493D484D
:10A68000002522C005608561C5613B490562C16046
:10A690000838FCF7D7FAFDF71FFDFDF701FEFDF7BF
:10A6A000DDFDFDF7E5FC052601223607D103304626
:10A6B000FCF719F9FEF756FAFDF7DEFBFBF71AFA7D
:10A6C000FBF7E8F90721B015FFF7D8FC2B4C0A215E
:10A6D000608A01224843E083170339463046FCF77D
:10A6E00002F92448C82226498830FDF74DF9254E45
:10A6F0006079002839D0A078002836D0FEF7E0FC39
:10A700006571FBF7DDFB20700F2809D9012239465E
:10A710003046FCF7E8F8FEF749FD0022394609E02B
:10A72000012251033046FCF7DEF8FEF73FFD002220
:10A73000012149033046FCF7D6F8FDF7EDFAE08B2E
:10A74000002801D0401EE0830F48E18B00780843C9
:10A75000CED10121C9023046FCF7BCF80028C7D190
:10A7600001210846FCF760FBC2E7FDF7D5FABFE719
:10A77000007C004070140020FFFF0000D400002087
:10A78000880C0020000400504200002010B586B064
:10A790001748FCF7DCF914216846FAF708FD15485C
:10A7A00000900320019000200290052069460007D8
:10A7B000FBF7D4FF69461048FBF7D0FF69460F4806
:10A7C000FBF7CCFF01210846FCF72EFBFF240134E8
:10A7D0002046FCF701FB0A49086804221043086080
:10A7E0002046FCF709FBFCF70FFB06B010BD00008C
:10A7F00070140020FFFF000000040050000800500B
:10A800000070004010B50122920218491848FBF769
:10A81000FFF91648174902888A4226D001807D2117
:10A82000C90081804910C1800A21018100211E22B6
:10A830004181D24382810122C2810184018241820D
:10A840008182C182018381831E23C3860223038701
:10A85000782343878287C28702464032118451841D
:10A860009184C183918000F02DF810BD500D00201F
:10A8700000FC0008AA550000F0B58C460025102603
:10A88000052109078E620E4C08E067467F5DE76090
:10A89000A768FF07FCD0E7681F706D1C8542F4DBDA
:10A8A0000020074606E0E760A568ED07FCD0E568F4
:10A8B0001D54401C9042F6D38E610020F0BD000074
:10A8C0000030014070B572B60124074DA402214644
:10A8D0002846FBF783F9002804D02246034928467E
:10A8E000FBF720FA62B670BD00FC0008500D002096
:10A8F000F0B50025102605279C463F070B46BE6293
:10A900000C4C06E0595DE160A168C907FCD0E16824
:10A910006D1C8542F6DB002007E06146095CE160C2
:10A92000A168C907FCD0E168401C9042F5D3BE6124
:10A930000020F0BD003001400000010203040005CA
:10A94000405C0000A05C0400C06C0800805C040057
:10A95000E03F1E00E07D1E0007A9022570889B884D
:10A960000A001600010006000100020087008D00A9
:10A970002D001A3152001A339A001A351D011A3768
:10A980006B003B31BE003B335E013B3596023B37EB
:10A99000000099599959EB518F421E45142E0080A1
:10A9A000EB51F5283333E13A703DE13AC235852B5E
:10A9B000C2353333C235C235AE47E13A5138A330E0
:10A9C00051380000000000000000010203040607E7
:10A9D0000809030406080C101820300000000001CC
:10A9E0000203040004AA0008000000202401000063
:10A9F0000C9A000828AB000824010020FC18000075
:10AA00001C9A000800000000000000000000000088
:10AA1000070400091E0805400826091040085608CA
:10AA2000054008261D040008BE1D040008BED8BC51
:10AA300040100800010000000000C84200000000B3
:10AA40000000000000000000000000000000000006
:10AA500000000000000000000000000000000000F6
:10AA600000000000000000000000000000000000E6
:10AA70005C12000000000000000000000000000068
:10AA800000000000000000000000000000000000C6
:10AA900000000000000000000000000000000000B6
:10AAA00000000000000000000000000000000000A6
:10AAB0000000000000000000000000000000000096
:10AAC00000000000020204000909010200810000E8
:10AAD0000000000001000000000100000000000074
:10AAE0000000000000000000000000000000000066
:10AAF0000000000000000000000000000000000056
:10AB00000000000000000000000000000000000045
:10AB10000000000000000000000000000000000035
:08AB200000002000000000000D
:04000005080050C1DE
:00000001FF
